:100000000C942A001895000018950000189500001F
:10001000189500001895000018950000189500002C
:10002000189500001895000018950000189500001C
:10003000189500001895000018950000189500000C
:1000400018950000189500001895000018950000FC
:10005000189500008FE58DBFC0E4E8E34E2E84E0E4
:100060008EBFD4E0F4E05F2EEEEFF3E0A0E6B0E068
:10007000A89584B7082E877F84BF88E1992781BD22
:1000800091BD88278D933197E9F783E389B980E0A3
:1000900080BD88E18AB966248FEF8ABBAFE6B0E005
:1000A000E0EFF3E00E947D010E945101A6E6B0E07E
:1000B000EAEFF3E00E947D010E9449010E94A6013F
:1000C00010ED0E94BE0110E00E94BE010E94A60138
:1000D00011ED0E94BE010E94DD01A0E6B0E01C937C
:1000E0000E94DD01A1E6B0E01C930E94DD01A2E6C2
:1000F000B0E01C930E94DD01AAE7B0E01C930E94CF
:10010000DD01A3E6B0E01C930E94DD01A4E6B0E0AF
:100110001C930E94DB01A5E6B0E01C930E94B50190
:10012000A0E6B0E09C910E943901A0E6B0E08C937B
:10013000A1E6B0E09C910E943901A1E6B0E08C9369
:10014000A2E6B0E09C910E943901A2E6B0E08C9357
:10015000A3E6B0E09C910E943901A3E6B0E08C9345
:10016000A4E6B0E09C910E943901A4E6B0E08C9333
:10017000A5E6B0E09C910E943901A5E6B0E08C9321
:100180000895A3E6B0E08C910E943201A3E6B0E0AE
:100190008C93A4E6B0E08C910E943201A4E6B0E01A
:1001A0008C93A5E6B0E08C910E943201A5E6B0E008
:1001B0008C930E94A60110ED0E94BE0114E00E94E3
:1001C000BE01A3E6B0E01C910E94BE01A4E6B0E02F
:1001D0001C910E94BE01A5E6B0E01C910E94BE01E8
:1001E0000E94B5010895A0E6B0E08C910E94320112
:1001F000A0E6B0E08C93A1E6B0E08C910E943201C1
:10020000A1E6B0E08C93A2E6B0E08C910E943201AE
:10021000A2E6B0E08C930E94A60110ED0E94BE0100
:1002200010E00E94BE01A0E6B0E01C910E94BE0159
:10023000A1E6B0E01C910E94BE01A2E6B0E01C91D4
:100240000E94BE010E94B5010895F894FFCF982F37
:1002500082958F70805D8D939F70905D9D938827B0
:100260008C9308954AE0082F0E9491010295802BFB
:100270000895892F8F70905110F0865FFCCF0895FC
:100280003197F1F70895689462F80895E89462F858
:100290000895E6E6F0E0A3E6B0E00E946D010E945A
:1002A000C100EFE6F0E0A0E6B0E00E945B010E9432
:1002B000F300ADE0BB27868197810E9487010D93F3
:1002C000838194810E9487010D93808191810E9496
:1002D00087010D930895ADE0BB27808191810E9435
:1002E00087010D93838194810E9487010D938681FC
:1002F00097810E9487010D9308950E9483010D92BA
:100300000020D9F70895C8953196002008958053AC
:1003100090530027813018F0065F8A95FBCF090FB4
:100320000895FF93881BF9E0001FFA9511F4FF91DF
:100330000895881F841B18F4840F8894F5CF0894BF
:10034000F3CFA998A898A198A0980895A09AA198E9
:1003500003D0A09801D0A19AEF93FF93E6E0F0E0DC
:100360000E944001FF91EF910895A09AA19AF4DFB5
:10037000A098989BFECFF0DFA198EECF0894111FB4
:1003800001C0110F69F0A09A18F40000A19802C0F2
:10039000A19A00C0E1DFA098989BFECFDDDFF1CFEE
:1003A000A09AA198D9DFA098989BFECFE89499993C
:1003B000689462F8D1CF089401C08894331F11E08B
:1003C000A09AA198C9DFA098989BFECFC5DF88941A
:1003D00099990894111FA0F7A09A379510F4A19845
:1003E00001C0A19AB9DFA098989BFECFB5DF089510
:1003F00031323A31363A3030000032362E30312E3A
:040400003131000096
:00000001FF
